:0A00000032C060C0FDCFFCCFFBCF83
:10000A00FACFF9CFF8CFF7CFEFC0F5CFF4CFF3CFD0
:10001A00F2CFF1CFF0CFEFCFEECFEDCF3B063B06DD
:10002A003B063B063B063B063B063B063B063C06BD
:10003A003C063C063C063C063C063C063C063C06A6
:10004A0052032E094105CC06EE07000000001200FB
:10005A007801260012008A0138000000F894EE2781
:10006A00ECBBF1E0FBBFEBBFE5BFF8E1F1BDE1BDE1
:10007A008DE0A2E0BB27ED938A95E9F780E094E052
:10008A00A0E6ED930197E9F7E8E5F0E0859195910F
:10009A00009761F0A591B59105901590BF01F00107
:1000AA0005900D920197E1F7FB01F0CFEFE5EDBF67
:1000BA00E4E0EEBFC0E6D1E088C3F5D36F936FB733
:1000CA006F937F938F939F936CB57DB585B780FBB4
:1000DA004EF4609372017093730165B76C7F62602E
:1000EA0065BF11C0609374017093750180917201AC
:1000FA0090917301681B790B609376017093770175
:10010A0065B7636065BF9F918F917F916F916FBF54
:10011A006F9115B71170113019F4689420F802C064
:10012A00E89420F821F821FE0CC0EAE4F0E0D3D4E8
:10013A00C4D3C8D328F0ECE4F0E0CDD4C6D308F495
:10014A0001C006C0689425F8E89420F8C2D3C4D345
:10015A0021FE05C0C8D3B9D310F422FE01C009C0DC
:10016A00E89424F8689422F8E894C1D3EAE0E0938A
:10017A00710121FE06C0B7D3A0D3A4D310F422FC88
:10018A0001C004C0E89424F8A7D3A3D321FE03C076
:10019A00AAD39BD308F005C0E89424F822F86894FF
:1001AA00A6D321FE04C023FE02C022FE01C01AC04B
:1001BA00E0916001A1D3A6D380D3A083B183E0915B
:1001CA006001EF5FE0936001A0916001A83011F433
:1001DA00689424F8A0916001A93018F0E8E0E0934F
:1001EA00600177D392D318955ED37894689426F8F1
:1001FA0010E0103148F492D36AD4DF019ED410F48F
:10020A008DD395D31F5FF5CFA0917101A13028F04E
:10021A00E0917101E150E093710177D318958DD384
:10022A00E4E5F0E08ED478948DD3A881A03148F427
:10023A008CD3EFEFFFEF92D394D3A0E0A08396D3B1
:10024A00F4CF96988E9AE8EEF3E094D38E98969A25
:10025A00E0B3E074E03409F08CC074D38ED348F470
:10026A008FD390D393D318F47CD3A1E0A0837ED309
:10027A00F5CF68D382D360F483D384D38ED330F49A
:10028A00E88190D3E759FE4FA1E0A0836FD3F2CF64
:10029A00A0916101A13011F4C09A01C0C098E09107
:1002AA006201E13011F4C19A01C0C198E091630181
:1002BA00E13011F4C29A01C0C298E0916401E130C0
:1002CA0011F4C39A01C0C398E0916501E13011F4B9
:1002DA00C49A01C0C498E0916601E13011F4C59A4C
:1002EA0001C0C598E0916701E13011F4A89A01C0F4
:1002FA00A898E0916801E13011F4A99A01C0A9987F
:10030A00E0916901E13011F4AA9A01C0AA98E0913A
:10031A006A01E13011F4AB9A01C0AB98E0916B012C
:10032A00E13011F4AC9A01C0AC98E0916C01E13073
:10033A0011F4AD9A01C0AD98E0916D01E13011F46C
:10034A00909A01C09098E0916E01E13011F4919A6F
:10035A0001C09198E0916F01E13011F4949A01C0C3
:10036A009498E0917001E13011F4959A01C0959842
:10037A006FCF96988E9AE0EDF7E0FCD28E98969A17
:10038A00E89426F8E0B3E074E03411F526FE1FC0C5
:10039A00D9D2F3D258F4F4D2F5D2F8D210F426FC1A
:1003AA0001C002C0D2D2C3D2E1D2F3CFCBD2E5D2BE
:1003BA0060F4E6D2E7D2F1D210F426FC01C003C001
:1003CA00F3D2F5D2B4D2D2D2F2CFE89426F8DACF69
:1003DA0096988E9AE0EDF7E0CDD2F894B3D2A88140
:1003EA00A03108F5E9D2BF01B0D271D3AFEFBFEFA8
:1003FA0076D3EA1BFB0BDB01B1D2A7D268D37E9777
:10040A0020F4A3D2EEE1F0E0A9D2DDD2E3D29DD26C
:10041A005ED3D0017BD3C8D2A05EBF4FA2D2E08107
:10042A007DD3A4D2DCCF8E98969A0000FECF1A9381
:10043A0010E010E01830F0F4E12FB4D2EF59FE4F7B
:10044A00E081E130A9F4E12F57D29CD29FD228F45F
:10045A00C4D2DF01C9D236D208F00AC0E12FC8D20D
:10046A00E12FACEBB1E09ED2EE0FFF1F8BD2C6D2CA
:10047A001F5FE0CF10E01830E0F4E12F93D2E75984
:10048A00FE4FE081E13099F4E12F36D27BD285D25A
:10049A0028F4A3D2DF01B4D2B7D208F008C0E12F02
:1004AA00E85FA6D2A12FB0E082D211D3A7D21F5FF4
:1004BA00E2CF9AD2ACD2A8D220F496D2ADD2A4D2AC
:1004CA0008F00FC0A0916101A13031F4A0919C0104
:1004DA00B0919D0132D309F002C0C09801C0C09A00
:1004EA0001C0C0989ED2A2D218F4A2D29FD208F01C
:1004FA000FC0E0916201E13031F4E0919E01F09188
:10050A009F01309709F002C0C19801C0C19A01C089
:10051A00C19893D28BD218F495D288D208F00FC022
:10052A00E0916301E13031F4E091A001F091A10181
:10053A00309709F002C0C29801C0C29A01C0C2989D
:10054A0086D274D218F488D271D208F00FC0E09122
:10055A006401E13031F4E091A201F091A3013097F6
:10056A0009F002C0C39801C0C39A01C0C39879D2E6
:10057A005DD218F47BD25AD208F00FC0E09165011F
:10058A00E13031F4E091A401F091A501309709F02E
:10059A0002C0C49801C0C49A01C0C4986CD246D2A1
:1005AA0018F46ED243D208F00FC0E0916601E13030
:1005BA0031F4E091A601F091A701309709F002C049
:1005CA00C59801C0C59A01C0C5985FD22FD218F448
:1005DA0061D22CD208F00FC0E0916701E13031F40A
:1005EA00E091A801F091A901309709F002C0A898FA
:1005FA0001C0A89A01C0A89852D218D218F454D2AD
:10060A0015D208F00FC0E0916801E13031F4E091B1
:10061A00AA01F091AB01309709F002C0A99801C074
:10062A00A99A01C0A998ECD1F2D14CD120F4E8D111
:10063A00F3D148D108F00FC0E0916901E13031F4FB
:10064A00E091AC01F091AD01309709F002C0AA988F
:10065A0001C0AA9A01C0AA98E4D12BD218F4E8D111
:10066A0028D208F00FC0E0916A01E13031F4E0913C
:10067A00AE01F091AF01309709F002C0AB9801C00A
:10068A00AB9A01C0AB98D9D114D218F4DBD111D2EC
:10069A0008F00FC0E0916B01E13031F4E091B00154
:1006AA00F091B101309709F002C0AC9801C0AC9A40
:1006BA0001C0AC98CCD1FDD118F4CED1FAD108F052
:1006CA000FC0E0916C01E13031F4E091B201F09198
:1006DA00B301309709F002C0AD9801C0AD9A01C0CC
:1006EA00AD98BFD1E6D118F4C1D1E3D108F00FC05B
:1006FA00E0916D01E13031F4E091B401F091B5017E
:10070A00309709F002C0909801C0909A01C0909861
:10071A00B2D1CFD118F4B4D1CCD108F00FC0E09146
:10072A006E01E13031F4E091B601F091B7013097F2
:10073A0009F002C0919801C0919A01C09198A5D17F
:10074A00B8D118F4A7D1B5D108F00FC0E0916F0164
:10075A00E13031F4E091B801F091B901309709F034
:10076A0002C0949801C0949A01C0949898D1A1D1DA
:10077A0018F49AD19ED108F00FC0E0917001E130CF
:10078A0031F4E091BA01F091BB01309709F002C04F
:10079A00959801C0959A01C0959810E0183068F4B0
:1007AA00E12FA8E7B1E0FED0EE0FFF1F13D1E12F32
:1007BA00A3D0E8D023D11F5FF1CF19910895E0E0CB
:1007CA00E8BBE5BBE0ECE2BB0895B7D0E6E5F0E0B4
:1007DA00B8D1E0E0E8BBEFE3E7BBE0E0E5BBEFE37D
:1007EA00E4BBE0ECE2BBE3E3E1BBE5E0E3BFE0E06E
:1007FA00E2BFEFBDE2E0EEBDE0E0EDBDECBDE7BD7E
:10080A00E6BDEBBDEABDE9BDE8BDE2BDE5BDE4BDBF
:10081A00E3BDEBB7E064EBBFE3E0E5BFE0E4EABFCA
:10082A00E1E0E9BFE0E8E8B9E0E0E0BF7894879B5F
:10083A00F6DC88D0A881A03188F493D00F01B4D017
:10084A00A05EBF4F57D1D001EC93B6D00F01BBD0F9
:10085A00AE0FBF1F4BD1D2D089D0ECCFE3EBE1BBB7
:10086A00E0ECE2BB25FE03C0AADFE89425F824FEEB
:10087A0004C023FE02C020FC01C00EC0E89420F888
:10088A00D6DDE89422F823F8979B02C0979902C014
:10089A00979A01C097980000E0917101E03009F43D
:1008AA008EDFE0CFFFCF0A92AA93BA93EA93FA9324
:1008BA00EFB7EA931A9310E00895A0917601B091E8
:1008CA0077010895AE17BF070895F7DFEA17FB0708
:1008DA000895E89421F80895E89422F823F8E0E0CE
:1008EA00E09360010895E2E5F0E0F5D0089523F879
:1008FA00E0E0E0936001EDCFAAE8B1E0F0E0EE0FAE
:10090A00FF1F0895EA0FFB1F08951991E991EFBFA0
:10091A00F991E991B991A99109900895E12FACE96A
:10092A00B1E0F0E0EE0FFF1FAE0FBF1F0895ED918B
:10093A00FD913197FE93EE930895219781E0A0E00F
:10094A00B0E00895E0E0E8830895E881ACEBB1E017
:10095A00F0E0EE0FFF1FAE0FBF1F0895ED93FC935B
:10096A000895E881F0E0EF59FE4F0895E881EF5FBE
:10097A00E8830895FA93EA939EC0A881A83008955F
:10098A00E881BACFAE0FBF1FA2D00895DF01E0E51C
:10099A00F0E0A1D0EA17FB070895DF01EEE4F0E0EA
:1009AA009AD090CFF0E00895A881B0E00895AA0FF8
:1009BA00BB1FA453BE4F0895E881ACEBB1E0F2DF50
:1009CA00EE0FFF1F9FCFE881A0E0B0E0EBDFEE0F54
:1009DA00FF1F089597DF0F010895E12FA8E7B1E0FF
:1009EA00E1DFEE0FFF1FCECFE0E5F0E074D008950F
:1009FA00ACE9B1E0D7DFEE0FFF1FECCFD001AECFED
:100A0A00EEE4F0E068D00895EA17FB070895A09194
:100A1A008A01B0918B010895A0917801B091790172
:100A2A000895A0918C01B0918D010895DDDFECCF7E
:100A3A00A0917A01B0917B010895A0918E01B091A5
:100A4A008F010895A0917C01B0917D010895A09134
:100A5A009001B09191010895A0917E01B0917F011A
:100A6A000895A0919201B09193010895A0918001F7
:100A7A00B09181010895A0919401B09195010895D2
:100A8A00A0918201B09183010895A0919601B0913D
:100A9A0097010895A0918401B09185010895A091CC
:100AAA009801B09199010895A0918601B0918701AA
:100ABA000895A6DF07CFE991F991309639F080EDD4
:100ACA0097E00197F1F7A8953197C9F70895ED9145
:100ADA00FC91119708950590F491E02D08951B2E2D
:100AEA00BF2FF12D1A2EAE2FE12D0895119602D0A7
:100AFA00FE2F1197E199FECFFF93FFB7F894AEBB93
:100B0A00BFBBE09AEDB3FFBFFF91089507D01196DE
:100B1A00EF93EF2F03D0EF9111970895E199FECF4C
:100B2A009FB7F894AEBBBFBBE09A8DB3E81719F034
:100B3A00EDBBE29AE19A9FBF089500240A160B06BC
:100B4A000895AC0FBD1F05900D928A95E1F708959F
:00000001FF
